:100000000C9469040C9491040C9491040C94910444
:100010000C9491040C9491040C9491040C9491040C
:100020000C9491040C9491040C942D0E0C949F0E3E
:100030000C9491040C9491040C9491040C949104EC
:100040000C9491040C94D4080C9491040C94910495
:100050000C9491040C9491040C9491040C94140845
:100060000C9491040C9491040C9491040C949104BC
:100070000C9491040C9491040C9491040C949104AC
:100080000C9472090C9491040C9491040C949104B6
:100090000C9491040C9491040C9491040C9491048C
:1000A0000C9491040C9491040C949104E904EC04D4
:1000B000DB04DF04E3040D050D050D05F004F40475
:1000C000F804FE0402050D050805040709070E07DC
:1000D000180722076C076C076C072C0736074007C8
:1000E0004A0757076C075F0700000000003E5B4FA0
:1000F0005B3E3E6B4F6B3E1C3E7C3E1C183C7E3C88
:10010000181C577D571C1C5E7F5E1C00183C180095
:10011000FFE7C3E7FF0018241800FFE7DBE7FF3025
:10012000483A060E2629792926407F050507407F93
:1001300005253F5A3CE73C5A7F3E1C1C08081C1C06
:100140003E7F14227F22145F5F005F5F06097F01FC
:100150007F006689956A606060606094A2FFA294E7
:1001600008047E040810207E201008082A1C0808B5
:100170001C2A08081E101010100C1E0C1E0C303803
:100180003E3830060E3E0E06000000000000005F04
:1001900000000007000700147F147F14242A7F2A20
:1001A00012231308646236495620500008070300E2
:1001B000001C2241000041221C002A1C7F1C2A082E
:1001C000083E080800807030000808080808000091
:1001D00060600020100804023E5149453E00427F05
:1001E000400072494949462141494D331814127F54
:1001F0001027454545393C4A4949314121110907F4
:100200003649494936464949291E00001400000074
:100210004034000000081422411414141414004146
:1002200022140802015909063E415D594E7C121103
:10023000127C7F494949363E414141227F4141413B
:100240003E7F494949417F090909013E41415173B6
:100250007F0808087F00417F41002040413F017F27
:10026000081422417F404040407F021C027F7F04EF
:1002700008107F3E4141413E7F090909063E415138
:10028000215E7F09192946264949493203017F0128
:10029000033F4040403F1F2040201F3F4038403F29
:1002A000631408146303047804036159494D43003F
:1002B0007F4141410204081020004141417F040276
:1002C000010204404040404000030708002054540D
:1002D00078407F28444438384444442838444428EB
:1002E0007F385454541800087E090218A4A49C783E
:1002F0007F0804047800447D40002040403D007F9A
:100300001028440000417F40007C047804787C0879
:100310000404783844444438FC182424181824244D
:1003200018FC7C08040408485454542404043F4432
:10033000243C4040207C1C2040201C3C4030403C61
:1003400044281028444C9090907C4464544C4400C1
:100350000836410000007700000041360800020125
:100360000204023C2623263C1EA1A161123A404011
:10037000207A38545455592155557941215454788F
:1003800041215554784020545579400C1E52721228
:1003900039555555593954545459395554545800B0
:1003A00000457C410002457D420001457C40F0292A
:1003B0002429F0F0282528F07C5455450020545479
:1003C0007C547C0A097F49324949493232484848BD
:1003D00032324A4848303A4141217A3A4240207804
:1003E000009DA0A07D39444444393D4040403D3CFF
:1003F00024FF2424487E4943662B2FFC2F2BFF0922
:1004000029F620C0887E0903205454794100004415
:100410007D413048484A32384040227A007A0A0A00
:10042000727D0D19317D2629292F28262929292673
:1004300030484D4020380808080808080808382FB8
:1004400010C8ACBA2F102834FA00007B0000081442
:100450002A142222142A14089500220095AA005575
:1004600000AAAA55AA55AA000000FF00101010FF0C
:1004700000141414FF001010FF00FF1010F010F013
:10048000141414FC001414F700FF0000FF00FF1404
:1004900014F404FC141417101F10101F101F141450
:1004A000141F00101010F0000000001F101010109A
:1004B0001F10101010F010000000FF10101010108E
:1004C00010101010FF10000000FF140000FF00FFCC
:1004D00000001F10170000FC04F414141710171468
:1004E00014F404F40000FF00F7141414141414148A
:1004F000F700F7141414171410101F101F141414FD
:10050000F4141010F010F000001F101F0000001F66
:1005100014000000FC140000F010F01010FF10FF99
:10052000141414FF141010101F00000000F010FF2E
:10053000FFFFFFFFF0F0F0F0F0FFFFFF0000000012
:1005400000FFFF0F0F0F0F0F38444438447C2A2A56
:100550003E147E02020606027E027E026355494177
:10056000633844443C04407E201E2006027E020282
:1005700099A5E7A5991C2A492A1C4C7201724C3096
:100580004A4D4D303048784830BC625A463D3E496D
:100590004949007E0101017E2A2A2A2A2A44445F11
:1005A000444440514A444040444A51400000FF0105
:1005B00003E080FF000008086B6B08361236243613
:1005C000060F090F06000018180000001010003078
:1005D00040FF0101001F01011E00191D1712003C00
:1005E0003C3C3C00000000000601150126013701DB
:1005F0004A015D01720188019F01B801D201EE013B
:100600000B022A024B026E029302BA02E4021003AA
:100610003F037003A403DC03170455049704DD04AF
:1006200027057505C80520067D06E0064907B807B9
:100630002D08A9082D09B9094D0AEA0A900B400CAA
:10064000FA0CC00D910E6F0F5A1053115B127213FA
:100650009A14D41520178018F519801B231DDE1E4F
:10066000B420A622B524E4263429A72B402E00313D
:10067000EA330037453ABC3D68414C456B49C84DAB
:1006800068524F57805C006210111213151617182C
:100690001A1C1D1F21232527292C2E3134373A3EC1
:1006A0004145494E52575C62686E757B838B939CC3
:1006B000A5AFB9C4D0DCE9F70000000200090F00C3
:1006C00000030401000C0000000000000000000016
:1006D00000000000000000F0F89C8E8783878E9C4D
:1006E000F8F00000FEFF0303030303070EFCF8000D
:1006F00000FEFF0303030303070EFCF80000FFFFE7
:1007000000000000000000FFFF0000FEFF83838365
:100710008383C7EE7C380000F8FC0E070303030751
:100720000EFCF800003F7FE0C08080C0E07F3FFF0C
:10073000FF01010101010101FFFF0000FFFF0C0C9F
:100740000C0C1C3E77E3C100007FFFC0C0C0C0C0DE
:10075000E0703F1F00001F3F70E0C0C0C0E0703F6E
:100760001F00007FFFC1C1C1C1C1E3773E1C000073
:100770001F3F70E0C0C0C0E0703F1F0000000000DD
:1007800001FFFF0100000000000000240027002AF4
:10079000002D003000D5F08D14A1C881CFD9F1AF64
:1007A00020001402130212021502070208020401BB
:1007B0000C0106010000003C0404040000000000DD
:1007C0000404043C000000784040400000000000A9
:1007D000404040780000000000C0E0207050103021
:1007E000E0C0000000000000000F1F383020203063
:1007F000180F00000000000000001030F08080D0D2
:1008000070100000000000000020382C06030F3894
:1008100030200000000408020110408040102040F9
:1008200080408008020401804020100201108010E6
:100830002040402000000000250028002B002E0052
:100840003100040404040403040502020202040348
:10085000020202020606060606060404020202045A
:10086000040301080B000202020100090400000158
:1008700002020000052400100105240101010424E6
:100880000206052406000107058103100040090443
:100890000100020A000000070502024000000705EF
:1008A00083024000000403090412010002EF020168
:1008B00040412336800001010203014172647569E1
:1008C0006E6F204C4C430041726475626F7900007A
:1008D000741511241FBECFEFDAE0DEBFCDBF11E0EB
:1008E000A0E0B1E0E8E1FCE202C005900D92A43581
:1008F000B107D9F726E0A4E5B1E001C01D92AF3001
:10090000B207E1F714E0C9E6D4E004C02197FE0184
:100910000E94FF15C836D107C9F70E94CF100C946A
:100920000A160C940000CF92DF92EF92FF920F9381
:100930001F93CF93DF936C017A018B01C0E0D0E06D
:10094000CE15DF0589F0D8016D918D01D601ED91AD
:10095000FC910190F081E02DC6010995892B11F4DD
:100960007E0102C02196ECCFC701DF91CF911F918C
:100970000F91FF90EF90DF90CF900895362F90E089
:10098000FC01E854F94F4491FC01EB5EF74F2491D0
:10099000FC01EE5BF74F8491882309F451C0442396
:1009A000E1F150E0FA013197EF30F105B0F5EA5A84
:1009B000FF4F0C94FF15909180009F7707C0909196
:1009C00080009F7D03C090918000977F909380006E
:1009D00024C094B59F7702C094B59F7D94BD1DC07F
:1009E000909190009F7707C0909190009F7D03C0E9
:1009F00090919000977F909390000FC09091C000CD
:100A00009F7703C09091C0009F7D9093C00005C068
:100A10009091C200977F9093C200E82FF0E0EE0F14
:100A2000FF1FEC5CF74FA591B4918FB7F894EC9150
:100A3000311103C020952E2301C02E2B2C938FBF84
:100A400008953FB7F8948091630190916401A0915B
:100A50006501B091660126B5A89B05C02F3F19F02E
:100A60000196A11DB11D3FBFBA2FA92F982F88272E
:100A7000820F911DA11DB11DBC01CD0142E0660F89
:100A8000771F881F991F4A95D1F708958FB12CB110
:100A900093B130E02095309520743327A90123E0ED
:100AA000559547952A95E1F7292F30E02095309507
:100AB000207133273595279535952795242B8095DB
:100AC000807F822B0895FC0121912EBD9C5F219196
:100AD0000DB407FEFDCF2EBDE817F907C1F70DB421
:100AE00007FEFDCF08952F923F924F925F926F9233
:100AF0007F928F929F92AF92BF92CF92DF92EF92AE
:100B0000FF920F931F93CF93DF9300D000D000D0BC
:100B1000CDB7DEB76A3091F4FC01E85EFB4F40814F
:100B200032972081318158E0459F200D311D1124DD
:100B300031832083329711821082E4C06D3009F432
:100B4000E1C0FC01E85EFB4FD0803297608071808D
:100B50001C017CEE271A7BEF370AD1012D913C91C5
:100B60000D2D10E0203831057CF0B6E0DB9E200D25
:100B7000311D1124F10131832083FC01E75EFB4F1D
:100B80004081411194C0BEC0F0E46F1671046CF74F
:100B9000A90175E0D79E400D511D112414161506AC
:100BA00024F7A80173E0440F551F7A95E1F7460D2D
:100BB000571D14161506CCF6E5E06E9FD0011124E2
:100BC000BA83A983490160E070E044244394512C26
:100BD0006530710541F0E981FA81E60FF71FE851B0
:100BE000FF4FE49101C0E0E05301F8E04E2F417067
:100BF000C42E9C828B824B8148194D1508F048C049
:100C0000A501F42EB42FBA19BD15D8F5AB81BC815E
:100C1000A038B10598F54034510580F5AF2DA69563
:100C2000A695A695EA2EF12CDA01A770BB27BE8304
:100C3000AD83D701B695BA2FAA27B795A795EB80B4
:100C4000FC80AE0DBF1DA80FB91F72010D8002C040
:100C5000EE0CFF1C0A94E2F7FE82ED82CC2031F00C
:100C60005496FC905497ED80EF2806C0ED80E094F8
:100C70005496FC905497EF205496EC924F5F5F4F40
:100C8000C0CF4B815C814F5F5F4F5C834B83B3CFA1
:100C9000E695F150A00EB11EF111A8CF6F5F7F4F06
:100CA000800E911E6630710509F092CF5ECF6AEF1B
:100CB0006003A001619F500D112440585F4F4217FF
:100CC000530704F5DC01ED91FC910190F081E02DDA
:100CD0006AE026960FB6F894DEBF0FBECDBFDF9157
:100CE000CF911F910F91FF90EF90DF90CF90BF9029
:100CF000AF909F908F907F906F905F904F903F90BC
:100D00002F90099426960FB6F894DEBF0FBECDBF84
:100D1000DF91CF911F910F91FF90EF90DF90CF90D7
:100D2000BF90AF909F908F907F906F905F904F900B
:100D30003F902F900895089580E090E008950E94DC
:100D40000516CF93DF9390E0FC01EB5EF74F249103
:100D5000FC01EE5BF74F8491882361F190E0880FEE
:100D6000991FFC01E957F84FC591D491FC01EC5C47
:100D7000F74FA591B491611109C09FB7F89488818C
:100D8000209582238883EC912E230BC0623061F47E
:100D90009FB7F8943881822F809583238883EC91C4
:100DA0002E2B2C939FBF06C08FB7F894E8812E2B73
:100DB00028838FBFDF91CF9108951F93CF93DF9347
:100DC000182FEB0161E00E94A106209711F460E06A
:100DD00004C0CF3FD10539F461E0812FDF91CF917D
:100DE0001F910C94BE04E12FF0E0E854F94FE49118
:100DF0004E2F50E0FA013197EF30F10508F06CC04A
:100E0000EB59FF4F0C94FF1584B5806884BDC7BDB6
:100E100068C084B5806284BDC8BD63C08091800015
:100E2000806880938000D0938900C093880059C067
:100E300080918000806280938000D0938B00C0936B
:100E40008A004FC080918000886080938000D0939A
:100E50008D00C0938C0045C0809190008068809385
:100E60009000D0939900C09398003BC0809190006F
:100E7000806280939000D0939B00C0939A0031C011
:100E800080919000886080939000D0939D00C093E3
:100E90009C0027C08091C00080688093C000809132
:100EA000C0008F7B8093C000C093CF001AC0809198
:100EB000C00080628093C000C093D00012C08091B7
:100EC000C20088608093C2008091C2008B7F8093B3
:100ED000C200C093D20005C0C038D1050CF07CCF51
:100EE00076CFDF91CF911F9108958F929F92AF920D
:100EF000BF92CF92DF92EF92FF926B017C010E9432
:100F000021054B015C01C114D104E104F104F1F0AD
:100F10000E942105DC01CB0188199909AA09BB09A6
:100F2000883E9340A105B10570F321E0C21AD108B3
:100F3000E108F10888EE880E83E0981EA11CB11C20
:100F4000C114D104E104F10419F7DDCFFF90EF9053
:100F5000DF90CF90BF90AF909F908F90089520E347
:100F600041E068E070E088E390E00E947A0B20E3C3
:100F700041E068E070E088E490E00E947A0B21E0B4
:100F800040E368E170E088E290E00E947A0B21E0A3
:100F900040E368E270E088E290E00E947A0B85EA24
:100FA00091E00E94630564EC79E080E090E00E94AB
:100FB000750782E090E0909305018093040190937F
:100FC00003018093020181E090E0909307018093F8
:100FD00006019093010180930001E4E7F1E01182A2
:100FE0001082138212821582148217821682118651
:100FF0001086138612861586148617861686118A21
:10100000108A089584E290E09093A6058093A50548
:1010100089E390E09093A8058093A70589E391E088
:101020000E94C20B0C94AF071F920F920FB60F9243
:1010300011242F933F938F939F93AF93BF938091EE
:10104000700190917101A0917201B0917301309182
:10105000620123E0230F2D3720F40196A11DB11D5D
:1010600005C026E8230F0296A11DB11D2093620141
:101070008093700190937101A0937201B0937301FA
:101080008091630190916401A0916501B091660126
:101090000196A11DB11D8093630190936401A093FB
:1010A0006501B0936601BF91AF919F918F913F9180
:1010B0002F910F900FBE0F901F901895CF92DF9237
:1010C000EF92FF920F931F93CF93E82FF0E0EF5929
:1010D000F74FC491E62FF0E0603330F4E857F94F52
:1010E000E4910E2F10E006C0EE0FFF1FE857FA4FF5
:1010F000059114916801E12CF12C60E074E284EF19
:1011000090E0A70196010E94AF15BA01A9014150D4
:101110005109610971094115510581E0680771059F
:1011200080F060E970ED83E090E0A70196010E94F5
:10113000AF15BA01A901415051096109710983E054
:1011400001C081E0C130C9F0C33031F59091910008
:10115000987F892B80939100509399004093980039
:10116000109361010093600181E080935F018091A1
:1011700071008260809371000FC090918100987F10
:10118000892B80938100509389004093880080913F
:101190006F00826080936F00CF911F910F91FF903D
:1011A000EF90DF90CF9008951F920F920FB60F929D
:1011B00011242F933F938F939F93AF93BF93EF93FC
:1011C000FF9380915801882309F44DC08091540108
:1011D00090915501A0915601B0915701892B8A2B0E
:1011E0008B2B51F180918D01E0918E01F0918F0157
:1011F0009081892780838091540190915501A0911D
:101200005601B0915701181619061A061B06A4F5C7
:101210008091540190915501A0915601B0915701D0
:101220000197A109B1098093540190935501A093AE
:101230005601B093570120C01092580180916F0061
:101240008D7F80936F0090918D01E0918E01F091E0
:101250008F018081282F30E0892F90E08095909534
:101260008223932308C080918D01E0918E01F0913B
:101270008F01908189278083FF91EF91BF91AF917A
:101280009F918F913F912F910F900FBE0F901F90C4
:101290001895E82FF0E0EF59F74FE491E13019F09D
:1012A000E33069F0089580916F008D7F80936F0027
:1012B00090918D01E0918E01F0918F0108C0109204
:1012C0005F0190918A01E0918B01F0918C01808106
:1012D000282F30E0892F90E08095909582239323EA
:1012E000808308951F920F920FB60F9211242F93AF
:1012F0003F934F935F936F937F938F939F93AF939E
:10130000BF93EF93FF9380915F01882349F0809111
:101310008A01E0918B01F0918C0190818927808373
:1013200080916801882309F493C080915B019091BA
:101330005C01A0915D01B0915E01892B8A2B8B2B02
:1013400009F486C080915B0190915C01A0915D01E0
:10135000B0915E010197A109B10980935B0190935F
:101360005C01A0935D01B0935E01892B8A2B8B2BCE
:1013700009F06EC0E0915901F0915A01BF016F5F11
:101380007F4F70935A01609359014491942F907F3D
:10139000842F8F70903819F40E944909EBCF90394F
:1013A00081F43296F0935A01E0935901FB01649164
:1013B000909190018917F0F667FDDCCF0E945E08DE
:1013C000D9CF903E29F410925A0110925901D2CFF0
:1013D000903F19F4109268013BC097FDCBCF329635
:1013E000F0935A01E0935901FB01249130E0342B32
:1013F000A0916001B09161010E94F0156C507E4F88
:101400008F4F9F4F28EE33E040E050E00E94CE1512
:1014100020935B0130935C0140935D0150935E012A
:1014200080915B0190915C01A0915D01B0915E01A2
:10143000892B8A2B8B2B61F481E090E0A0E0B0E057
:1014400080935B0190935C01A0935D01B0935E017A
:10145000FF91EF91BF91AF919F918F917F916F918C
:101460005F914F913F912F910F900FBE0F901F9062
:101470001895FC0180918901811103C08FEF9FEFC6
:1014800008959FB7F89482E08093E9002091F200DC
:1014900030E01216130614F421E030E02115310576
:1014A00059F0289884E6809388018091F100808328
:1014B0008091F200882319F09FBFC90108958BE63F
:1014C0008093E800F9CF2FB7F89483E08093E90088
:1014D0009091E800892F807295FF04C09091F200EE
:1014E00080E4891B2FBF0895CF93DF931F92CDB760
:1014F000DEB76983DC01ED91FC910280F381E02D80
:1015000041E050E0BE016F5F7F4F09950F90DF9182
:10151000CF91089583E08093E9008091F2008823C1
:1015200019F08AE38093E80008950E94630A90E02E
:101530000895CF93DF931F92CDB7DEB7FC0184856A
:10154000958597FD05C02FEF3FEF358724870BC0AA
:10155000CE0101960E94390A019719F4898190E021
:1015600002C08FEF9FEF0F90DF91CF9108950F93FF
:101570001F93CF93DF931F92CDB7DEB78C01FC0191
:101580008485958597FF0EC0CE0101960E94390A89
:10159000019719F4298130E002C02FEF3FEFF801E5
:1015A00035872487F801848595850F90DF91CF9149
:1015B0001F910F910895FC018485958597FD0BC0BF
:1015C0009FB7F89482E08093E9008091F2009FBF7A
:1015D00090E0019608959FB7F89482E08093E90027
:1015E0008091F2009FBF90E008958F929F92AF92FA
:1015F000BF92CF92DF92EF92FF920F931F93CF9300
:10160000DF935C016B017A0180910F01882309F45B
:101610005BC080918901882309F456C080918701BD
:1016200080FF05C08091E00082608093E000E701C8
:1016300010E00AEF83E0882E9AE3992E2097D9F1E3
:101640000E94630A81110AC0015009F43DC061E0A3
:1016500070E080E090E00E947507F0CF282F30E026
:10166000C217D3070CF48C2F4FB7F8948092E9007F
:101670009091E80095FF1DC0282F30E0C21BD30BCE
:10168000F601982F915020F081918093F100FACFCC
:10169000C20ED31E112319F09092E80009C0809168
:1016A000E80085FD06C09092E80011E0209709F05F
:1016B00010E04FBFC3CF1111C3CF5D9884E6809374
:1016C00086011E141F0444F081E090E0F50193832D
:1016D000828380E090E001C0C701DF91CF911F912C
:1016E0000F91FF90EF90DF90CF90BF90AF909F90C1
:1016F0008F900895EF92FF920F931F93CF93DF93F4
:10170000EC01C40FD11DDB01A20FB11D01E010E0FF
:101710008C179D0784F59B0177FF24C020E030E003
:1017200021C0241735072CF580389105C8F4422FC5
:10173000469546954695FC0150E8459FE00DF11D04
:101740001124EF56FE4FA90147705527780102C0BA
:10175000EE0CFF1C4A95E2F7A7015489452B448BF8
:101760002F5F3F4FAD01A134B105DCF240E450E002
:10177000D8CF0196CDCFDF91CF911F910F91FF90E0
:10178000EF900895009769F0FC0101900020E9F7BF
:101790003197AF01481B590BBC0181E991E00C94D2
:1017A000930480E090E0089520E085EA91E0B22F74
:1017B000B111BFEFFC010024B193B193B193B19388
:1017C0000394D1F708952F923F924F925F926F92B8
:1017D0007F928F929F92AF92BF92CF92DF92EF92C1
:1017E000FF920F931F93CF93DF93CDB7DEB7279769
:1017F0000FB6F894DEBF0FBECDBFA22EB12C9C0158
:101800002A0D3B1D37FDB3C0803891050CF0AFC0E9
:101810009B01205F3F4F2035310508F0A8C0DB0158
:1018200077FF04C0AA27BB27A61BB70BA770BB274F
:101830009B0177FF02C0295F3F4FF3E03595279565
:10184000FA95E1F777FF08C02150310968E070E0B0
:101850004B018A1A9B0AD401B9017695762F662727
:1018600077956795680F791F290102E0400E511C9A
:10187000E12CF12CE8E0F0E04F018A1A9B0A9F82EC
:101880008E822F3F0FEF300774F42F5F3F4FEA0C2B
:10189000FB1C60587F4F2415350509F468C02830BB
:1018A000310579F764C03B0110E8610E711C8B01B2
:1018B0000B5D1D4F6C011B821A828A809B808A14EB
:1018C0009B041CF7E0E8CE16D104F9F2D7FC41C026
:1018D0002F3FFFEF3F0709F447C0EA81FB81EE0D80
:1018E000FF1DE40FF51FE491480186189708860E46
:1018F000971E2E2E312CF1010A2E02C0EE0FFF1F73
:101900000A94E2F7FD83EC83F4012080EC81FD81F1
:10191000E229FD83EC833C80F40130821097C9F00A
:1019200027303105B1F0EA81FB81EE0DFF1DE40F98
:10193000F51FE491F0E01F010E8002C0359427945A
:101940000A94E2F7F8019080F101E9294F01F801CA
:101950008082EA81FB813196FB83EA830F5F1F4F10
:10196000FFEFCF1ADF0AA9CF1097E9F6F2CF27963B
:101970000FB6F894DEBF0FBECDBFDF91CF911F91A0
:101980000F91FF90EF90DF90CF90BF90AF909F901E
:101990008F907F906F905F904F903F902F90089521
:1019A000CF93DF9390919001923009F46EC0C82FCD
:1019B000292F30E0F901EF59F74FD491F901E9549B
:1019C000FA4F80839F5F9093900161E00E94A1068F
:1019D000D13019F0D33039F158C0109280001092F4
:1019E00081008091810088608093810080918100D6
:1019F0008160809381008C2F90E0FC01EE5BF74FBB
:101A0000E491F0E0EE0FFF1FEC5CF74F259134916D
:101A100030938F0120938E01FC01EB5EF74F849190
:101A200080938D0132C010929000109291008091AD
:101A300091008860809391008091910081608093F3
:101A400091008C2F90E0FC01EE5BF74FE491F0E009
:101A5000EE0FFF1FEC5CF74F2591349130938C0112
:101A600020938B01FC01EB5EF74F849180938A01F8
:101A700080919001882321F06CE380E00E945E0851
:101A800080E0DF91CF910C944909DF91CF910895C7
:101A90008091AF0581110DC082E08093AB0584E099
:101AA0008093AC051092AE051092AD0581E0809355
:101AB000AF058BEA95E0089540910D0650910E0612
:101AC00020910B0630910C0642175307B4F4909105
:101AD000E8009570E1F39091E80092FD19C08093C1
:101AE000F10080910D0690910E0601968F73992753
:101AF000892B19F48EEF8093E80080910D06909168
:101B00000E06019690930E0680930D0681E00895CF
:101B100080E00895CF92DF92EF92FF920F931F9390
:101B2000CF93DF931F92CDB7DEB7182F062FE42E89
:101B3000862F880F8E5F99830E945C0D83E00E9440
:101B40005C0DF12EC12E9981D92E8C2D8F19801705
:101B500098F4F601E7FE02C0849101C080810E94E2
:101B60005C0D182F80E00E945C0D8123FFEFCF1ADF
:101B7000DF0A8111EACF01C081E00F90DF91CF91A0
:101B80001F910F91FF90EF90DF90CF900895DF921B
:101B9000EF92FF920F931F93CF93DF93D82E8A017A
:101BA0007B01E40EF51EEB01CE15DF0571F0D7FECB
:101BB00003C0FE01849101C088810E945C0D2196C2
:101BC0008111F2CF8FEF9FEF01C0C801DF91CF915C
:101BD0001F910F91FF90EF90DF900895615030F0CA
:101BE0002091F100FC0120830196F8CF289884E62B
:101BF0008093880108950F931F93CF93DF931F92D3
:101C0000CDB7DEB782E0898342E450E063E678E056
:101C100080E80E94C70D0E94480DDC0112960D91CC
:101C20001C9113970115110569F0D801ED91FC91F4
:101C30000280F381E02DBE016F5F7F4FC8010995DF
:101C400097FF07C089810F90DF91CF911F910F916E
:101C50000895F80100851185E5CF1F920F920FB608
:101C60000F9211248F939F938091E1009091E10056
:101C7000937F9093E10083FF0FC01092E90091E001
:101C80009093EB001092EC0092E39093ED00109291
:101C9000890198E09093F00082FF20C093E0909338
:101CA000E9009091F200992319F09AE39093E800EB
:101CB00090918601992339F09091860191509093EB
:101CC0008601992389F190918801992339F09091A7
:101CD0008801915090938801992341F184FF10C0AD
:101CE0008091E2008E7E81608093E2008091E1002D
:101CF0008F7E8093E100809187018E7E806111C08C
:101D000080FF16C08091E2008E7E80618093E200A9
:101D10008091E1008E7E8093E100809187018E7E2C
:101D200081608093870104C05D9ACDCF289AD6CF79
:101D30009F918F910F900FBE0F901F9018951F923B
:101D40000F920FB60F921124CF92DF92EF92FF9273
:101D50000F931F932F933F934F935F936F937F93B3
:101D60008F939F93AF93BF93EF93FF93CF93DF93A3
:101D7000CDB7DEB76C97DEBFCDBF1092E900809182
:101D8000E80083FFEDC168E0CE0145960E94EE0DAC
:101D900082EF8093E8008D8987FF05C09091E8006D
:101DA00090FFFCCF03C09EEF9093E800982F9076B1
:101DB00009F0C6C09E892F89188D91110CC08038FA
:101DC00029F480910A068093F10002C01092F1007C
:101DD0001092F10048C1422F50E0512B913051F444
:101DE000811141C14130510509F03DC180910A0680
:101DF0008D7F0BC0933061F4811135C141305105A5
:101E000009F031C180910A06826080930A062BC1D5
:101E1000953041F48091E80080FFFCCF206820934A
:101E2000E30021C1963009F05FC0EB8CFC8C10926E
:101E3000E90010920E0610920D06123091F51092E4
:101E40000C0610920B060E94FB0D99E0BE016F5F1D
:101E50007F4FDB01E92F1D92EA95E9F799831A83F9
:101E600091E09E8390EA98879AEF998720910D06DA
:101E700030910E06275F3F4F3C832B838D8310925A
:101E8000E90010920E0610920D06F0920C06E092F8
:101E90000B0649E050E080E00E94C70D0E94FB0D58
:101EA000E2C0F0920C06E0920B060E94480DDC01A5
:101EB0001296ED90FC901397E114F10409F4C0C060
:101EC000D701ED91FC910480F581E02DBE016B5EA0
:101ED0007F4FC7010995009719F00CF0C4C0C7C027
:101EE000F701E084F184E8CF973009F4C0C098305E
:101EF00021F481E08093F100B6C0993009F0B3C0BD
:101F0000837009F0B4C0E3E3F1E081E021E036E35F
:101F10009081992361F08093E9002093EB009191E7
:101F20009093EC003093ED008F5F873089F78EE758
:101F30008093EA001092EA008F898093890193C010
:101F40008B8D9C8D1092E90010920E0610920D065A
:101F500090930C0680930B06898D811156C08E8953
:101F60009D89913A59F4813209F081C047E050E0EF
:101F700068E071E080E00E94C70D75C0913209F001
:101F800076C0833289F4888D90E0982F88272F8936
:101F9000822BA0E0B0E08093100190931101A093F8
:101FA0001201B09313015FC0803269F48091E800A0
:101FB00082FFFCCF67E088E091E00E94EE0D8BEF9E
:101FC0008093E80006C0823209F04DC08F8980936B
:101FD0000F0180910906882319F0EEEFFAE002C0A4
:101FE000E0E0F8E08091080190910901A0910A01D8
:101FF000B0910B01803B9440A105B10509F07BC075
:1020000080910F0180FF93C076C00E94480DDC01D3
:1020100012960D911C9113970115110541F1D801EC
:10202000ED91FC910190F081E02DBE016B5E7F4F40
:10203000C8010995811117C0F80100851185ECCF01
:10204000113009F44EC0133091F48F89882309F4BC
:1020500045C0823081F440E867E087EC98E00E9458
:102060008A0D882321F08EEF8093E80079C081E209
:102070008093EB0075C0813029F440E86BE08BEB76
:1020800098E0EDCF833099F70E94480DDC0112965D
:10209000ED90FC9013978E010F5F1F4F6801E114C4
:1020A000F10479F0D701ED91FC910680F781E02DE4
:1020B000B801C7010995080F111DF701E084F184EB
:1020C000EECFD8011C92F60101900020E9F731977C
:1020D000BF016C197D0940E0C601C1CF65EA78E017
:1020E00002C069EA78E06115710509F2FB014491CB
:1020F00050E080E840CF0FB6F894A895809160003A
:10210000886180936000109260000FBEA895EE3F3A
:102110002AE0F20739F08091FE0A9091FF0A91833C
:102120008083A1CF1092FF0A1092FE0A9CCFEE3F4F
:102130008AE0F80731F0808191819093FF0A8093C3
:10214000FE0A87E797E7918380839BE088E10FB6DB
:10215000F894A895809360000FBE9093600083CFA1
:102160006C960FB6F894DEBF0FBECDBFDF91CF9156
:10217000FF91EF91BF91AF919F918F917F916F915F
:102180005F914F913F912F911F910F91FF90EF9091
:10219000DF90CF900F900FBE0F901F901895CF93A8
:1021A000DF93CDB7DEB7A1970FB6F894DEBF0FBEB1
:1021B000CDBF789484B5826084BD84B5816084BDD0
:1021C00085B5826085BD85B5816085BD80916E00D5
:1021D000816080936E001092810080918100826006
:1021E0008093810080918100816080938100809143
:1021F0008000816080938000809191008260809354
:102200009100809191008160809391008091900075
:102210008160809390008091C10084608093C100B0
:102220008091C10082608093C1008091C100816073
:102230008093C1008091C30081608093C30080912E
:10224000C00082608093C0008091C2008160809352
:10225000C20080917A00846080937A0080917A0035
:10226000826080937A0080917A00816080937A0006
:1022700080917A00806880937A0010928901109290
:102280000A06109287018091D70081608093D70061
:1022900080EA8093D80089B5806189BD89B5826064
:1022A00089BD09B400FEFDCF61E070E080E090E000
:1022B0000E9475078091D8008F7C80618093D80040
:1022C0008091E000807F8093E0008091E1008E7E2D
:1022D0008093E1008DE08093E200559A209AEEEF22
:1022E000FFE7859194918B3F9C4D19F481E0809399
:1022F00009061FB7F89480916901811127C0E3E5B1
:10230000F8E08491E6E2F8E09491E82FF0E0EE0F37
:10231000FF1FE957F84FA591B491EC91E92321F4FF
:1023200061E081E10E94BE0461E081E10E94A106BA
:102330008CB580618CBD8CB580648CBD61E08FE014
:102340000E94A10661E080E10E94A10680916901DE
:102350008F5F809369011FBF02EA17E0F801849143
:1023600031966491882329F00E5F1F4F0E94A106C9
:10237000F5CF61E086E00E94BE0461E070E080E09D
:1023800090E00E94750760E086E00E94BE046AE06B
:1023900070E080E090E00E94750761E086E00E94B6
:1023A000BE04EEE4F8E0E491F0E0EE0FFF1FEC5C19
:1023B000F74F8591949190936F0180936E01E1E2C4
:1023C000F8E0E491E0936D01E6E4F8E0E491F0E0F8
:1023D000EE0FFF1FEC5CF74F8591949190936C0189
:1023E00080936B01E9E1F8E0E491E0936A018CB538
:1023F0008C7F8CBD8DB581608DBDE0916E01F091BB
:102400006F01908180916D01982B9083A0916B0159
:10241000B0916C012C9190916A01909592239C93BC
:102420009081809589238083E5E9F7E027E0E23A0F
:10243000F20749F084918EBD00000DB407FEFDCF78
:102440008EB53196F3CFE0916B01F0916C019081E4
:1024500080916A01892B8083E0916E01F0916F0178
:10246000908180916D0180958923808380916400A3
:102470008160809364008091640082608093640036
:10248000809164008068809364008091640080641F
:1024900080936400809165008160809365000E9454
:1024A000460587FF1AC080E094E01EBC00000DB412
:1024B00007FEFDCF2EB50197C1F760E070E08AE01E
:1024C0000E94DD0660E070E08BE00E94DD0660E0C7
:1024D00070E089E00E94DD06FFCF0EEE1FEFA8E15D
:1024E000FA2ECC24CA94D12C8F2D801BB601681BE8
:1024F00071098AE00E94DD066FEF70E08BE00E94B8
:10250000DD066FEF70E089E00E94DD060E94D40BCB
:1025100028E547ED56E0B80184E190E00E94E30B26
:1025200085EA91E00E9463056BE170E080E090E055
:102530000E947507003F31F46AEF70E080E090E0A0
:102540000E9475070F5F1F4F0931110569F66EEE86
:1025500072E080E090E00E9475076FEF70E08AE023
:102560000E94DD066FEF70E08BE00E94DD066FEFEA
:1025700070E089E00E94DD0685E00E94D00C8DE0CD
:102580000E94D00C1092680182E090E00E94A71592
:10259000882369F080916400877F80936400809134
:1025A0006500877F8093650081E0809367010E94CA
:1025B000D40B8AE08093970184E680939A01FAE035
:1025C0004F2E512C612C712C79E3272E312CE3E016
:1025D0008E2E912C2FB7F8948091700190917101FB
:1025E000A0917201B09173012FBF2091A30122230A
:1025F00091F020919B01382F321B3093A401209140
:102600009801309199012F5F3F4F309399012093AA
:1026100098011092A30140919F015091A0016091F7
:10262000A1017091A20184179507A607B7077CF452
:10263000481B423008F450C283B7817F83BF83B701
:10264000816083BF889583B78E7F83BF45C2209109
:102650009A01AC01BD01420F511D611D711D4093D6
:102660009F015093A0016093A1017093A2018093F8
:102670009B0190939C01A0939D01B0939E0181E0EA
:102680008093A3010E94D40B8AE290E09093A60568
:102690008093A5051092A8051092A70584E491E007
:1026A0000E94C20BC0900601D09007010D2C000CB7
:1026B000EE08FF08F7FE26C0E0919101F09192012B
:1026C0000190F081E02D6DE281E991E009952227EA
:1026D0003327A9012C193D094E095F0919A28E0162
:1026E0000F5D1F4FCA01B901A30192010E94CE15CF
:1026F000605DF80162938F01211531054105510597
:1027000089F715C0A701960119A28E010F5D1F4F11
:10271000CA01B901A30192010E94CE15605DF801C2
:1027200062938F01211531054105510589F7C801D3
:102730000E94C20B0E94460585FF09C080910401DA
:1027400090910501019790930501809304010E94E7
:10275000460586FF09C0809104019091050101960C
:1027600090930501809304010E94460587FF09C0EC
:10277000809102019091030101979093030180934E
:1027800002010E94460584FF09C0809102019091D8
:102790000301019690930301809302010E94460574
:1027A00083FF34C0E0910401F091050131978091DD
:1027B00002019091030101979F01220F331FE20F45
:1027C000F31FE80FF91FEE0FFF1FEC58FE4F80813B
:1027D0009181892BD9F42091060130910701318331
:1027E0002083809100019091010101969093010155
:1027F000809300012130310519F482E090E002C09D
:1028000081E090E090930701809306010E944605C5
:1028100080910401909105011816190634F081E0A9
:1028200090E09093050180930401809104019091C0
:102830000501049724F09092050180920401809193
:102840000201909103011816190634F081E090E01E
:102850009093030180930201809102019091030102
:10286000049724F0909203018092020144E7A42E81
:1028700041E0B42E08E210E038E0C32ED12CE12C68
:10288000F12CF501EE0DFF1D8081918181309105C4
:1028900021F420E145EF57E005C0029739F420E12B
:1028A00045ED57E0B601C8010E94E30BF2E0EF0EE0
:1028B000F11C20E1C20ED11C36E0E316F10409F749
:1028C000005F1F4F86E0A80EB11C08351105A1F668
:1028D000809174019091750120917C0130917D016E
:1028E0008217930759F42091840130918501821752
:1028F000930721F4892B11F00E940208809178013E
:102900009091790120917C0130917D01821793078C
:1029100059F420918001309181018217930721F4AD
:10292000892B11F00E940208809174019091750129
:1029300020917601309177018217930759F4209105
:102940007801309179018217930721F4892B11F0D6
:102950000E94020880917A0190917B0120917C0174
:1029600030917D018217930759F420917E013091B7
:102970007F018217930721F4892B11F00E9402082E
:102980008091800190918101209182013091830199
:102990008217930759F420918401309185018217A1
:1029A000930721F4892B11F00E9402088091740191
:1029B0009091750120917A0130917B0182179307E4
:1029C00059F420918001309181018217930721F4FD
:1029D000892B11F00E940208809176019091770175
:1029E00020917C0130917D018217930759F4209149
:1029F0008201309183018217930721F4892B11F012
:102A00000E940208809178019091790120917E01C5
:102A100030917F018217930759F4209184013091FE
:102A200085018217930721F4892B11F00E94020877
:102A300080910001909101010A9784F0E0E3F0E0B9
:102A4000F093A605E093A5053092A8052092A7056E
:102A50008CE491E00E94C20B0E94AF0720E341E0AA
:102A600068E070E088E390E00E947A0B20E341E0A8
:102A700068E070E088E490E00E947A0B21E040E397
:102A800068E170E088E290E00E947A0B21E040E388
:102A900068E270E088E290E00E947A0B60910201A7
:102AA0007091030184E0660F771F8A95E1F7685003
:102AB0007109809104019091050124E0880F991F0C
:102AC0002A95E1F720E145EB57E048960E94E30B99
:102AD00085EA91E00E94630580E090E0892B09F48B
:102AE00079CD0E94000070CDE9EBF5E013821282EF
:102AF00088EE93E0A0E0B0E084839583A683B7835B
:102B000088E191E0918380838FEF9FEF95878487A1
:102B1000E1E9F1E0138212828AE291E091838083FD
:102B20008CE3868380E1818710861782168617865C
:102B3000108A118A128A1092A6051092A505109289
:102B4000A8051092A70581E08093A9050895F99939
:102B5000FECF92BD81BDF89A992780B50895052EC4
:102B600097FB1EF400940E94C61557FD07D00E94E3
:102B7000CE1507FC03D04EF40C94C6155095409525
:102B8000309521953F4F4F4F5F4F08959095809519
:102B9000709561957F4F8F4F9F4F0895A1E21A2E38
:102BA000AA1BBB1BFD010DC0AA1FBB1FEE1FFF1FF1
:102BB000A217B307E407F50720F0A21BB30BE40B41
:102BC000F50B661F771F881F991F1A9469F7609588
:102BD0007095809590959B01AC01BD01CF01089542
:102BE000A29FB001B39FC001A39F700D811D11244E
:102BF000911DB29F700D811D1124911D0895EE0F3E
:102C0000FF1F0590F491E02D099481E090E0F89485
:082C10000C940A16F894FFCFA2
:102C1800010002000200010000E1000000000000C5
:102C2800FFFFFFFF00000000740AF50A950A8A0AF0
:102C3800DB0A990AB70A00000000730593049C0692
:102C48009B0600C18081000000596F752057696E8E
:102C580021212100506C6179657220005469652139
:042C68002121000026
:00000001FF
